S02B0000433A2F576F726B2F736F6674776172652F4F70656E424C542F5461726765742F44656D6F2F41524DEF
S1134000E40100209B4100000D4600000D46000025
S11340100D4600000D4600000D4600000D46000050
S11340200D4600000D4600000D4600000D46000040
S11340300D4600000D4600000D46000089460000B4
S11340400D4600000D4600000D4600000D46000020
S11340500D4600000D4600000D4600000D46000010
S11340600D4600000D4600000D4600000D46000000
S11340700D4600000D4600000D4600000D460000F0
S11340800D4600000D4600000D4600000D460000E0
S11340900D4600000D4600000D4600000D460000D0
S11340A00D4600000D4600000D4600000D460000C0
S11340B00D4600000D4600000D4600000D460000B0
S11340C00D4600000D4600000D4600000D460000A0
S11340D00D4600000D4600000D4600000D46000090
S11340E00D4600000D4600000D4600000D46000080
S10740F0EE11AA55CA
S11340F42B49072291438D462A482B492B4A00F029
S113410439F82B482B492C4A00F034F82B482C4915
S11341142C4A00F02FF82C482C492D4A00F02AF898
S11341242C482D492D4A00F025F82D482D492E4AB6
S113413400F020F82D482E49002200F026F82D48DE
S11341442D49091A082903DB0022026004300160A6
S11341541E481F49884205D00268043003B49047BE
S113416403BCF7E700208646EC4600200021234ADE
S11341749047FEE7884207D0521A05D003780130ED
S11341840B700131013AF9D17047884202D00270B0
S11341940130FAE770471A481A490160A8E7000099
S11341A4E40100200C660000000000200000002050
S11341B40C4200000C4200001C6300000C6600006A
S11341C400000020000000201C6300001C630000A9
S11341D41C6300001C6300001C6300001C630000DB
S11341E41C6300001C6300000C6600000000002037
S11341F46400002064000020E40000209D450000C9
S10B420408ED00E00040000099
S113420C80B500AF024B9847024B984700BF80BD66
S113421C4D4200002D44000080B500AF024B98477E
S113422C024B984700BF80BD99420000A94400008E
S113423C80B500AF014B984700BF80BDC54F00004F
S113424C98B500AF0A480B4B98470B48094B984755
S113425C03214FF04020094B9847094B98470146DE
S113426C60234FF461420748074CA04700BF98BD38
S113427C01000010614F0000010000207D4B000084
S113428C0152000000C000404555000080B500AF4D
S113429C254B1B78002B15D12448254B98470346F6
S11342AC012B3FD1214B1B78002B3BD0214B984742
S11342BC0246214B1A601C4B01221A701F4B002220
S11342CC1A702FE01D4B1B780133184A13441846FF
S11342DC174B98470346012B19D1184B1B78013304
S11342ECDAB2164B1A70114B1A78144B1B789A428B
S11342FC18D10D4B00221A700C4B5B78FF2B11D18B
S113430C0A4B9B78002B0DD10D4B98470AE0094BB7
S113431C98470246084B1B6864339A4202D9024BF5
S113432C00221A7000BF80BD000000200400002091
S113433C5143000075460000480000204C0000204A
S113434C3D42000080B584B000AF786009480A4B48
S113435C9847F860FB68B3F1FF3F05D0FB68DAB20D
S113436C7B681A70012300E0002318461037BD4601
S113437C80BD00BF00C000405557000080B586B01A
S113438C00AF0423FB6010237B603DE00823BB607B
S113439C34E07B680133642202FB03F27968BB6866
S11343AC0B440133B2FBF3F3FB75FB7D402B22D999
S11343BCFB7D4B2B1FD87A68BB6813440133102246
S11343CCB2FBF3F103FB01F3D31A002B13D1BB683B
S11343DC032B01D8BB68FB607A68BB6813440133B8
S11343EC1022B2FBF3F33B613B1D19460A480B4BFD
S11343FC984701230CE0BB68013BBB60BB68002BF6
S113440CC7D17B68013B7B607B68002BBED100234A
S113441C18461837BD4680BD00000440055B0000FB
S113442C90B587B000AF1348134B9847032113483A
S113443C134B98471348104B98471348134B984702
S113444C134B98471048134B984740F267637B60B3
S113445C40F2FF73BB600823FB6008233B613A1DE9
S113446C0223012108480C4CA04700BF1C37BD4651
S113447C90BD00BF08000020614F00000070004098
S113448CCD4A00000001100000000440B5590000A2
S113449C89430000B55A00004D5D000090B589B009
S11344AC00AF02210F48104B9847F86101231A46BC
S11344BCFB691340002B10D03B46BB6107F108028B
S11344CC012301210748094CA0473B78FF2B04D159
S11344DC7B78002B01D1064B984700BF2437BD468F
S11344EC90BD00BF00000440595C000059600000FE
S11344FC3D42000080B500AF0648074B98470121A8
S113450C0648074B9847002201210448054B98475D
S113451C00BF80BD20000020614F0000005002400D
S113452C254B0000814A000080B582B000AF134BCC
S113453C98477860124B1B687A68D31AB3F5FA7FE4
S113454C18D3104B1B78002B08D10E4B01221A7078
S113455C012201210C480D4B984707E0094B00221E
S113456C1A70002201210848084B9847044A7B68BA
S113457C136000E000BF0837BD4680BD75460000DF
S113458C500000205400002000500240814A0000DA
S113459C80B500AF044B9847044B9847044B98479D
S11345AC044B9847FAE700BFC54500000D420000D4
S11345BC354500002542000080B500AF0448054B8A
S11345CC9847054B9847054B984700BF80BD00BFE3
S11345DC8003C001E54F00000145000015460000B2
S11345EC80B483B000AF78603960034A7B68136091
S11345FC024A3B681360FEE7580000205C00002070
S113460C80B400AFFEE700BF80B500AF094B9847FC
S113461C0246094BA3FB02239B091846074B9847F8
S113462C074B9847074B98470020074B984700BF08
S113463C80BD00BF01520000D34D6210C95400006C
S113464C91540000AD5400005946000080B483B06E
S113465C00AF7860034A7B68136000BF0C37BD461B
S113466C80BC70476000002080B400AF024B1B6814
S113467C1846BD4680BC70476000002080B400AF73
S113468C044B1B680133034A136000BFBD4680BC56
S113469C704700BF6000002080B483B000AF786026
S11346AC7B68B3F1402F43D07B68264A93423FD0BA
S11346BC7B68254A93423BD07B68244A934237D08B
S11346CC7B68234A934233D07B68224A93422FD08F
S11346DC7B68214A93422BD07B68204A934227D093
S11346EC7B681F4A934223D07B681E4A93421FD097
S11346FC7B681D4A93421BD07B681C4A934217D09B
S113470C7B681B4A934213D07B681A4A93420FD09E
S113471C7B68194A93420BD07B68184A934207D0A2
S113472C7B68174A934203D07B68164A934201D1A3
S113473C012300E00023DBB218460C37BD4680BCD5
S113474C704700BF008005400050004000900540B9
S113475C0060004000A005400070004000B005401F
S113476C0040024000C005400050024000D005400B
S113477C0060024000E005400070024000F005407B
S113478C00D003400000064080B584B000AFF86050
S113479C0B467A60FB72F868244B98470346002B4F
S11347AC03D1E4212248234B98477B68002B09D082
S11347BC7B68012B06D07B68022B03D0E6211C48B6
S11347CC1C4B9847FB6803F5806319467B6803F020
S11347DC0103002B06D0FB6803F580631A68FB7A8F
S11347EC134306E0FB6803F580631B68FA7AD24333
S11347FC13400B60FB6803F5846319467B6803F074
S113480C0203002B06D0FB6803F584631A68FB7A59
S113481C134306E0FB6803F584631B68FA7AD243FE
S113482C13400B6000BF1037BD4680BDA546000089
S113483C1C630000ED45000080B584B000AFF86047
S113484C7A603B600B46FB72F868874B98470346CB
S113485C002B04D14FF4DD718448854B98477B6859
S113486C012B0DD07B68022B0AD07B68042B07D05C
S113487C7B680C2B04D04FF4DF717C487C4B98473D
S113488C3B68082B16D03B680A2B13D03B680C2BC7
S113489C10D03B68092B0DD03B680B2B0AD03B681E
S11348AC0D2B07D03B68002B04D040F2C5116F4888
S11348BC6F4B9847FB6803F5A06319467B6803F0BC
S11348CC0103002B06D0FB6803F5A0631A68FB7A7E
S11348DC134306E0FB6803F5A0631B68FA7AD24322
S11348EC13400B60FB6803F2045319467B6803F016
S11348FC0203002B06D0FB6803F204531A68FB7AFC
S113490C134306E0FB6803F204531B68FA7AD243A0
S113491C13400B60FB6803F5A16319467B6803F035
S113492C0403002B06D0FB6803F5A1631A68FB7A19
S113493C134306E0FB6803F5A1631B68FA7AD243C0
S113494C13400B60FB6803F5A36319467B6803F003
S113495C0803002B06D0FB6803F5A3631A68FB7AE3
S113496C134306E0FB6803F5A3631B68FA7AD2438E
S113497C13400B60FB6803F20C5319463B6803F0BD
S113498C0103002B06D0FB6803F20C531A68FB7A64
S113499C134306E0FB6803F20C531B68FA7AD24308
S11349AC13400B60FB6803F5A26319463B6803F0E4
S11349BC0203002B06D0FB6803F5A2631A68FB7A8A
S11349CC134306E0FB6803F5A2631B68FA7AD2432F
S11349DC13400B60FB6803F2145319463B6803F055
S11349EC0403002B06D0FB6803F214531A68FB7AF9
S11349FC134306E0FB6803F214531B68FA7AD243A0
S1134A0C13400B60FB6803F21C5319463B6803F01C
S1134A1C0803002B06D0FB6803F21C531A68FB7ABC
S1134A2C134306E0FB6803F21C531B68FA7AD24367
S1134A3C13400B60FB6803F5A56319463B68002B18
S1134A4C06D1FB6803F5A5631A68FB7A134306E0E9
S1134A5CFB6803F5A5631B68FA7AD24313400B6019
S1134A6C00BF1037BD4680BDA54600001C63000086
S1134A7CED45000080B582B000AF78600B46FB704A
S1134A8C1346BB7078680B4B98470346002B04D134
S1134A9C4FF451710848094B9847FB789B001A4610
S1134AAC7B6813441A46BB78136000BF0837BD46B5
S1134ABC80BD00BFA54600001C630000ED4500004E
S1134ACC90B583B000AF78600B46FB7078680D4BE3
S1134ADC98470346002B04D14FF464710A480B4BDE
S1134AEC9847FB78022219467868094B9847F9785D
S1134AFC082304227868074CA04700BF0C37BD4636
S1134B0C90BD00BFA54600001C630000ED450000ED
S1134B1C954700004548000090B583B000AF78601D
S1134B2C0B46FB7078680D4B98470346002B04D159
S1134B3C40F204410A480B4B9847FB780122194672
S1134B4C7868094B9847F978082301227868074C50
S1134B5CA04700BF0C37BD4690BD00BFA546000062
S1134B6C1C630000ED45000095470000454800001B
S1134B7C90B583B000AF78600B46FB7078680D4B32
S1134B8C98470346002B04D140F21F510A480B4BA3
S1134B9C9847FB78022219467868094B9847F978AC
S1134BAC082301227868074CA04700BF0C37BD4688
S1134BBC90BD00BFA54600001C630000ED4500003D
S1134BCC954700004548000080B582B000AF78607E
S1134BDC7B68462B04D94FF4D5712348234B984753
S1134BEC7B68042B06D1224A214B1B6843F4803387
S1134BFC136035E07B68052B06D11D4A1C4B1B68E2
S1134C0C43F4003313602BE07B68062B06D1184A5F
S1134C1C174B1B6843F48023136021E07B680F2B34
S1134C2C06D1144A134B1B6843F00203136017E0BC
S1134C3C7B680F2B0AD97B682F2B07D80E4A7B680D
S1134C4C103B012101FA03F3136009E07B682F2B5D
S1134C5C06D90A4A7B68303B012101FA03F313603D
S1134C6C00BF0837BD4680BD88630000ED450000D9
S1134C7C24ED00E010E000E000E100E004E100E0DD
S1134C8C80B582B000AF78607B68462B04D94FF4B2
S1134C9CF7712348234B98477B68042B06D1224A8F
S1134CAC214B1B6823F48033136035E07B68052BA0
S1134CBC06D11D4A1C4B1B6823F4003313602BE0F4
S1134CCC7B68062B06D1184A174B1B6823F48023E8
S1134CDC136021E07B680F2B06D1144A134B1B681D
S1134CEC23F00203136017E07B680F2B0AD97B684F
S1134CFC2F2B07D80E4A7B68103B012101FA03F3D2
S1134D0C136009E07B682F2B06D90A4A7B68303B79
S1134D1C012101FA03F3136000BF0837BD4680BDBF
S1134D2C88630000ED45000024ED00E010E000E095
S1134D3C80E100E084E100E080B483B000AF7860EF
S1134D4C7B685E4A934200F0AF807B685C4A934276
S1134D5C00F0AA807B685B4A934200F0A5807B68D4
S1134D6C594A934200F0A0807B68584A934200F061
S1134D7C9B807B68564A934200F096807B68554A28
S1134D8C934200F091807B68534A934200F08C80EC
S1134D9C7B68524A934200F087807B68504A934266
S1134DAC00F082807B684F4A93427DD07B684E4AE8
S1134DBC934279D07B684D4A934275D07B684C4AB8
S1134DCC934271D07B684B4A93426DD07B684A4ABC
S1134DDC934269D07B68494A934265D07B68484AC0
S1134DEC934261D07B68474A93425DD07B68402BE9
S1134DFC5AD07B68B3F1102F56D07B68424A934249
S1134E0C52D07B68414A93424ED07B68404A9342CD
S1134E1C4AD07B683F4A934246D07B683E4A9342D1
S1134E2C42D07B68B3F1101F3ED07B683B4A93425F
S1134E3C3AD07B683A4A934236D07B68394A9342DB
S1134E4C32D07B68384A93422ED07B68374A9342DF
S1134E5C2AD07B68364A934226D07B68354A9342E3
S1134E6C22D07B68344A93421ED07B68334A9342E7
S1134E7C1AD07B68324A934216D07B68314A9342EB
S1134E8C12D07B68304A93420ED07B68B3F1202F4A
S1134E9C0AD07B682D4A934206D07B68082B03D03A
S1134EAC7B682B4A934201D1012300E00023DBB23F
S1134EBC18460C37BD4680BC704700BF010010007B
S1134ECC0200100000011000000210000004100089
S1134EDC00011010000210100004101000401010FB
S1134EEC00501020010000200200002004000020CB
S1134EFC08000020100000202000002040000020AA
S1134F0C8000002000010020004000100010101050
S1134F1C000110208000003010000030000100104F
S1134F2C00020010100000102000001020000030BF
S1134F3C01001010020010100400101008001010D2
S1134F4C01000010020000100400001001001020E9
S1134F5C0010100080B582B000AF78607868124BF6
S1134F6C98470346002B04D14FF4FC710F48104BA7
S1134F7C98477B681B0F0F4A52F8233018467B68FE
S1134F8C1B0F0C4A52F823301A687B6899B27B6861
S1134F9C1B0C03F01F0301FA03F31343036000BF5C
S1134FAC0837BD4680BD00BF454D0000606400005D
S1134FBCED450000F863000080B400AF014B024AD9
S1134FCC1A60FEE70CED00E00400FA0501387FF4EA
S1134FDCFDAF704700BF00BF80B586B000AF7860EE
S1134FEC794B1B6803F0E043002B06D0764B1A6810
S1134FFC764B1340B3F1805F03D17B68002BC0F276
S113500CDE80734B1B683B61724B1B68FB603B6916
S113501C43F400633B613B6923F480033B61FB680D
S113502C43F40063FB606A4A3B691360694AFB689A
S113503C13603B6903F00203002B04D07B6803F07C
S113504C0203002B09D03B6903F00103002B2BD086
S113505C7B6803F00103002B26D17B6863F0030308
S113506C3A6913403B615A4A3B691360FB68002B55
S113507C09DAFB6803F07003302B0CD0FB6803F0E7
S113508C7003702B07D0FB68002B09DB3B6903F022
S113509C3003302B04D14FF480504F4B984703E02E
S11350AC4FF400204C4B98473B6923F45F5323F097
S11350BC30033B617A6843F2F07313403A6913434B
S11350CC3B61FA68454B1340FB607A68444B1340D0
S11350DCFA681343FB607B68DB0003F04003FA6857
S11350EC1343FB603F4B40221A60FB68002B06DA2B
S11350FC384AFB681360364A3B69136005E0344A4E
S113510C3B691360334AFB6813601020324B984799
S113511C3B6923F0F86323F003033B617A68324B59
S113512C13403A6913433B61FB6823F0FC53FB6067
S113513C7B6803F0FC53FA681343FB607B6803F051
S113514C8043002B0ED03B6943F480033B61FB6826
S113515C23F48003FB607A68244B1340FA681343EE
S113516CFB6003E0FB6823F08043FB607B6803F483
S113517C0063002B19D14FF400437B6108E01C4BF6
S113518C1B6803F04003002B06D17B69013B7B6158
S113519C7B69002BF3D100E000BF3B6923F400636F
S11351AC3B61FB6823F40063FB60094A3B691360B1
S11351BC084AFB6813601020074B984700E000BFB7
S11351CC1837BD4680BD00BF00E00F400000FF70E3
S11351DC60E00F4070E00F40D94F00008FDFFF7F7D
S11351EC3020008058E00F400300C007000040400E
S11351FC50E00F4080B485B000AF944B1B68FB604B
S113520C934B1B687B607B68002B03DA7B6803F091
S113521C700302E0FB6803F03003202B45D0202BF5
S113522C04D8002B09D0102B10D079E0602B6FD050
S113523C702B71D0302B67D072E0FB689B0903F0A4
S113524C1F03844A52F82330BB606BE0824B1B680B
S113525C03F0E043002B06D07F4B1A687F4B1340BE
S113526CB3F1805F02D17E4BBB601DE07A4B1A68B0
S113527C7A4B13407B4A934204D1774B1B689BB205
S113528C022B0BD0744B1A68744B1340764A93421E
S113529C07D1714B1B689BB2002B02D1734BBB60C3
S11352AC02E0734BBB603DE03CE06B4B1B6803F0CE
S11352BCE043002B06D0684B1A68684B1340B3F1DB
S11352CC805F02D16B4BBB601DE0634B1A68634B70
S11352DC1340644A934204D15F4B1B689BB2022B6C
S11352EC0BD05D4B1A685D4B13405F4A934207D158
S11352FC594B1B689BB2002B02D15F4BBB6002E085
S113530C5E4BBB600EE00DE047F23053BB6009E02E
S113531C4FF48003BB6005E04FF40043BB6001E035
S113532C00238EE07B68002B04DA7B6803F40063B3
S113533C002B07D07B68002B47DBFB6803F400636E
S113534C002B42D14E4B1B683B60434B1B6803F054
S113535CE043002B06D0404B1A68404B1340B3F18A
S113536C805F0FD13B685B09C3F308030233BA684F
S113537C02FB03F23B6803F01F030233B2FBF3F3AB
S113538CBB600EE03B685B09C3F30803BA6802FB1D
S113539C03F23B6803F01F0301335B00B2FBF3F32E
S11353ACBB603B6803F48043002B02D0BB685B08F2
S11353BCBB603B6803F40043002B02D0BB689B0822
S11353CCBB60FB6843F48003FB60FB6803F480035D
S11353DC002B35D07B68002B29DA7B6803F08043E3
S11353EC002B1AD07B68002B04DA7B6803F400636F
S11353FC002B07D07B68002B0FDBFB6803F40063E6
S113540C002B0AD1BB685A007B689B0D03F07F0309
S113541C0133B2FBF3F3BB6012E07B68DB0D03F0EA
S113542C3F030133BA68B2FBF3F3BB6008E0FB68DB
S113543CDB0D03F00F030133BA68B2FBF3F3BB606B
S113544CBB6818461437BD4680BC704760E00F40FB
S113545C70E00F400464000000E00F400000FF7097
S113546CC0E1E4000000011000000310001BB700B1
S113547C0024F40070383900C0C62D0000093D002A
S113548C64E00F4080B400AF044A044B1B6843F043
S113549C0503136000BFBD4680BC704710E000E0FC
S11354AC80B400AF044A044B1B6843F0020313603E
S11354BC00BFBD4680BC704710E000E080B582B0F0
S11354CC00AF78607B68002B03D07B68B3F1807FDE
S11354DC03D9D0210548064B9847064A7B68013B03
S11354EC136000BF0837BD4680BD00BFCC6400000C
S11354FCED45000014E000E080B483B000AF7860A8
S113550C7B680A4A934207D07B68094A934203D0CA
S113551C7B68084A934201D1012300E00023DBB2EB
S113552C18460C37BD4680BC704700BF00C0004015
S113553C00D0004000E0004080B586B000AFF860B9
S113554CB9607A603B60F868444B98470346002B7B
S113555C04D140F20D114248424B98477B68002B12
S113556C04D14FF487713E483E4B98473E4B1B6821
S113557C03F0E043002B1ED03B4B1A683B4B13400B
S113558CB3F1805F17D0384B1A68384B1340384A44
S113559C934204D1344B1B689BB2022B0BD0324B7D
S11355AC1A68324B1340334A934206D12E4B1B6874
S11355BC9BB2002B01D1102300E008237A6802FB74
S11355CC03F2BB689A4204D940F20F112448254BCC
S11355DC9847F868284B98477B681A01BB689A422D
S11355EC0CD9FB6830331A46FB6830331B6843F024
S11355FC200313607B685B087B6008E0FB68303336
S113560C1A46FB6830331B6823F020031360BB6815
S113561CDA007B68B2FBF3F301335B087B61FB6854
S113562C24331A467B699B091360FB6828331A469A
S113563C7B6903F03F031360FB682C331A463B6809
S113564C1360FB6818331A4600231360F8680B4B7D
S113565C984700BF1837BD4680BD00BF05550000F4
S113566C38650000ED45000000E00F400000FF70BD
S113567C0000011000000310E95600008D560000D4
S113568C80B582B000AF78607868114B98470346B8
S113569C002B04D14FF4CF710E480F4B98477B6805
S11356AC2C331A467B682C331B6843F010031360AD
S11356BC7B6830331A467B6830331B6843F4407381
S11356CC43F00103136000BF0837BD4680BD00BF23
S11356DC0555000038650000ED45000080B582B02A
S11356EC00AF78607868154B98470346002B04D1BB
S11356FC4FF4DF711248134B984700BF7B68183383
S113570C1B6803F00803002BF8D17B682C331A4672
S113571C7B682C331B6823F0100313607B683033D5
S113572C1A467B6830331B6823F4407323F001035F
S113573C136000BF0837BD4680BD00BF055500008F
S113574C38650000ED45000080B582B000AF78608C
S113575C78680D4B98470346002B04D140F209415D
S113576C0A480B4B98477B6818331B6803F01003EB
S113577C002B02D17B681B6801E04FF0FF33184605
S113578C0837BD4680BD00BF0555000038650000D4
S113579CED45000080B483B000AF78607B680A4AA2
S11357AC934207D07B68094A934203D07B68084A2A
S11357BC934201D1012300E00023DBB218460C37DD
S11357CCBD4680BC704700BF00000440001004407C
S11357DC0020044080B485B000AF78607B680D4A2B
S11357EC934208D00C4A934208D00C4A934208D1F5
S11357FC3723FB6008E03823FB6005E03923FB60AA
S113580C02E04FF0FF33FB60FB6818461437BD46CB
S113581C80BC704700100440002004400000044089
S113582C80B586B000AF78607B6823F47F6323F087
S113583C0F031846194B984703467B617B69B3F1F8
S113584CFF3F03D1F9211648164B9847164B1B689A
S113585C7A69303A012101FA02F213403B613B6947
S113586C002B02D07869114B98477B681B68002386
S113587CBB6002E0BB680133BB60BB68042BF9DD81
S113588C7B681B68FB603B69002B02D07869084B72
S113589C9847FB6818461837BD4680BDE157000091
S11358ACA4650000ED45000004E100E08D4C00000F
S11358BCD54B000080B485B000AF786039607B684C
S11358CC3A681A600023FB6002E0FB680133FB605A
S11358DCFB68042BF9DD00BF1437BD4680BC704750
S11358EC80B586B000AFF860B9607A6000237B6144
S11358FC1EE07B695A1C7A611A46FB6813441B78B8
S113590C3B617A697B689A420BDA7B695A1C7A612F
S113591C1A46FB6813441B781B021A463B69134353
S113592C3B61BB681A1DBA6039691846044B984729
S113593C7A697B689A42DCDB00BF1837BD4680BDB0
S113594CC158000080B586B000AFF860B9607A60C9
S113595C00237B611DE0BB681A1DBA601846114B0D
S113596C984738617B695A1C7A611A46FB68134460
S113597C3A69D2B21A707A697B689A4209DA7B69FD
S113598C5A1C7A611A46FB6813443A69120AD2B259
S113599C1A707A697B689A42DDDB00BF1837BD4602
S11359AC80BD00BF2D58000080B584B000AF786076
S11359BC7868384B98470346002B04D140F2D91130
S11359CC3548364B984701217868354B984700BFCA
S11359DC7B6820331846334B9847034603F4004343
S11359EC002BF5D17B682433B02118462C4B9847F7
S11359FC7B68343300211846294B98477B6838332D
S1135A0C00211846264B98470123FB6014E000BF85
S1135A1C7B6820331846234B9847034603F4004312
S1135A2C002BF5D17B682033FA68114618461C4BC1
S1135A3C9847FB680133FB60FB68202BE7DD7B6830
S1135A4C24330C211846164B98470123FB6014E0B1
S1135A5C00BF7B6820331846124B9847034603F467
S1135A6C0043002BF5D17B682033FA6811461846A5
S1135A7C0B4B9847FB680133FB60FB68202BE7DD7D
S1135A8C7B6804331846074B984700BF1037BD4654
S1135A9C80BD00BFA1570000A4650000ED450000C7
S1135AACC15800002D58000080B582B000AF78605A
S1135ABC78680C4B98470346002B04D140F23A21EA
S1135ACC09480A4B98477868094B9847034623F0D2
S1135ADC010319467868074B984700BF0837BD4641
S1135AEC80BD00BFA1570000A4650000ED45000077
S1135AFC2D580000C158000080B584B000AF786008
S1135B0C396078684C4B98470346002B04D14FF40A
S1135B1C59714A484A4B98473B68002B04D140F2D0
S1135B2C65314648464B98473B681B68012B03D9A3
S1135B3C3B681B68102B04D940F26B313F48404B37
S1135B4C98473B685B68002B03D03B685B68082B69
S1135B5C04D94FF45C713948394B98473B689B68BE
S1135B6C002B03D03B689B68042B04D940F275319D
S1135B7C3248334B98473B68DB68B3F5806F03D8E6
S1135B8C3B68DB68002B04D140F27B312B482C4B57
S1135B9C984778682B4B9847F860FB6843F04103AF
S1135BAC19467868284B98473B685B68013B1B0394
S1135BBC03F4E043BB603B681B68013B1B0203F42A
S1135BCC7063BA681343BB603B689B68013B9B01E1
S1135BDCDBB2BA681343BB603B68DB68013B03F080
S1135BEC3F03BA681343BB607B680C33B96818462F
S1135BFC154B98477B6803F118023B68DB68013B43
S1135C0C9B0903F00F03194610460F4B9847FB688A
S1135C1C23F04003FB60FB6803F00103002B03D06B
S1135C2CFB6823F00103FB60F9687868064B98471E
S1135C3C00BF1037BD4680BDA1570000A46500000D
S1135C4CED4500002D580000C158000080B584B00B
S1135C5C00AF78600B46FB707868344B984703466A
S1135C6C002B04D140F292513148324B9847FB78C7
S1135C7C032B52D801A252F823F000BF995C000008
S1135C8CB55C0000DB5C0000015D00007B68043344
S1135C9C1846294B9847F8607B6804336FF01F0152
S1135CAC1846264B98473BE07B6803F580731846EF
S1135CBC214B9847F8607B6803F5827318461E4B9A
S1135CCC984703461B04FA681343FB6028E07B687F
S1135CDC03F590731846184B9847F8607B6803F5E6
S1135CEC92731846144B984703461B04FA681343E3
S1135CFCFB6015E07B6803F5B07318460E4B9847B0
S1135D0CF8607B6803F5B27318460B4B984703464F
S1135D1C1B04FA681343FB6002E00023FB6000BF22
S1135D2CFB6818461037BD4680BD00BFA157000064
S1135D3CA4650000ED4500002D580000C15800007A
S1135D4C80B588B000AFF860B9607A60FB7000234E
S1135D5CFB74F868784B98470346002B04D140F247
S1135D6C5F617648764B9847BB68202B02D8BB689A
S1135D7C002B04D14FF4CC617048714B9847FB78DD
S1135D8C002B13D0FB78012B10D0FB78022B0DD0F9
S1135D9CFB78032B0AD0FB78012B07D0FB78042B60
S1135DAC04D040F266616548654B984700BFFB68B8
S1135DBC20331846634B9847034603F40043002BE7
S1135DCCF5D17B681B68B3F5006F05D27B689B68C3
S1135DDC03F00403002B02D00123BB7401E0002365
S1135DECBB749323FB8300233B830023FB8200239C
S1135DFCBB820023BB8300237B83FB78042B00F240
S1135E0C1D8101A252F823F0295E00003D5E0000C2
S1135E1C4B5E0000515E0000735E0000BB8A43F4CD
S1135E2C8073BB824FF40053FB820123FB7423E089
S1135E3CBB8A43F48073BB820023FB821CE00023E7
S1135E4CFB8219E04FF40053FB824FF48053BB8266
S1135E5C4FF6FF73BB8341F6FF737B83FB8B43F0DD
S1135E6C4003FB8308E04FF40053FB824FF4905340
S1135E7CBB820123FB7400BF7B689B6803F008039F
S1135E8C002B17D0BB7C002B0AD07B685B68BB83D0
S1135E9C7B685B681B0C9BB2C3F30C037B8309E02C
S1135EAC0023BB837B685B689BB29B009BB2C3F3F0
S1135EBC0C037B837B689B6803F02803282B05D198
S1135ECC7B8B6FEA43436FEA53437B837B689B680A
S1135EDC03F01803182B03D17B8B43F480437B838F
S1135EEC7B689B6803F03803002B07D0BB8A43F410
S1135EFC8053BB82FB8B43F04003FB83FB8B43F04F
S1135F0C2003FB83BB7C002B1ED07B681B689AB2DE
S1135F1C3B8B13433B837B681B681B0C9BB2C3F307
S1135F2C0C039AB2FB8A1343FB82FB8A6FEA83430A
S1135F3C6FEA9343FB8218E0A1570000A4650000AC
S1135F4CED4500002D5800007B681B689BB29B003C
S1135F5C9BB2C3F30C039AB2FB8A1343FB82FB8AF6
S1135F6C6FEA43436FEA5343FB827B68DB689BB263
S1135F7C03F00F039AB2BB8A1343BB827B689B6802
S1135F8C03F40073002B03D1BB8A43F08003BB8260
S1135F9C7B689B6803F00103002B03D0BB8A43F49A
S1135FAC0063BB827B689B6803F00203002B03D065
S1135FBCBB8A43F48063BB82FB7C002B09D07B68D7
S1135FCC1869FB683C3319467B68DB681A461D4B21
S1135FDC9847FB682433FA8B114618461A4B98479A
S1135FECFB682833BA8B11461846174B9847FB6845
S1135FFC2C337A8B11461846134B9847FB68303375
S113600C3A8B11461846104B9847FB683433FA8A7E
S113601C114618460C4B9847FB683833BA8A11461C
S113602C1846094B9847FB6803F12002BB6803F040
S113603C3F0319461046044B984700E000BF203735
S113604CBD4680BDED580000C158000080B588B035
S113605C00AFF860B9607A60FB70F868A54B98479C
S113606C0346002B04D140F2C171A348A34B9847BB
S113607CBB68202B02D8BB68002B04D140F2C27140
S113608C9D489E4B98477323FB83FB78002B03D0CE
S113609CFB8B43F00803FB83FB688433FA8B1146B8
S11360AC1846974B9847FB6803F18002BB6803F0D2
S11360BC3F0319461046924B984700BFFB68803348
S11360CC1846904B9847034603F40043002BF5D134
S11360DCFB68883318468B4B98470346BB83FB6895
S11360EC8C331846874B984703467B83FB68903365
S11360FC1846844B984703463B83FB6894331846F5
S113610C804B98470346FB82FB68983318467D4BBB
S113611C98470346BB827B6800229A60BB8A03F4CF
S113612C8073002B04D1FB8A03F40053002B09D198
S113613CBB8A03F48073002B0AD0FB8A03F400534C
S113614C002B05D17B689B6843F040027B689A6006
S113615CFB8A03F48043002B0FD0FB8A1A046A4B8E
S113616C13403A8B13431A467B681A607B689B680E
S113617C43F004027B689A6005E0FB8A9B10C3F32E
S113618C0A027B681A60BB8A03F48043002B05D097
S113619C7B689B6843F480727B689A60BB8A03F4C7
S11361AC8053002B4DD0FB8A03F48043002B1BD06F
S11361BC7B8B1A04544B1340BA8B13431A467B68DB
S11361CC5A607B685B686FF06042934205D17B68D0
S11361DC9B6803F04003002B1ED17B689B6843F043
S11361EC08027B689A6017E07B8B9B10C3F30A024E
S11361FC7B685A607B685B6840F2FF72934205D1FE
S113620C7B689B6803F04003002B05D17B689B687B
S113621C43F008027B689A60B7F91A30002B05DA50
S113622C7B689B6843F028027B689A607B8B03F441
S113623C8043002B05D07B689B6843F018027B6875
S113624C9A60BB8A03F40063002B05D07B689B68BF
S113625C43F001027B689A60BB8A03F48063002BD1
S113626C05D07B689B6843F002027B689A60B7F99F
S113627C1430002B36DABB8A03F00F027B68DA6029
S113628C7B689B6803F04003002B09D17B68186979
S113629CFB689C3319467B68DB681A461B4B984792
S11362ACFB68843304211846154B9847FB6803F1AB
S11362BC8002BB6803F03F0319461046104B984705
S11362CC00BFFB68803318460E4B9847034603F413
S11362DC0043002BF5D17B689B6843F080027B68FC
S11362EC9A6002E07B680022DA6000BF2037BD466A
S11362FC80BD00BFA1570000A4650000ED4500005F
S113630CC15800002D5800000000FF1F5159000017
S113631C433A2F576F726B2F736F66747761726584
S113632C2F4F70656E424C542F5461726765742FF5
S113633C44656D6F2F41524D434D335F4C4D335378
S113634C5F454B5F4C4D3353383936325F43726F74
S113635C7373776F726B732F50726F672F696465E9
S113636C2F2E2E2F6C69622F6472697665726C699C
S113637C622F6770696F2E6300000000433A2F5739
S113638C6F726B2F736F6674776172652F4F7065C4
S113639C6E424C542F5461726765742F44656D6F53
S11363AC2F41524D434D335F4C4D33535F454B5F3F
S11363BC4C4D3353383936325F43726F7373776F86
S11363CC726B732F50726F672F6964652F2E2E2F8B
S11363DC6C69622F6472697665726C69622F696E7E
S11363EC746572727570742E6300000000E10F40C6
S11363FC04E10F4008E10F4040420F0000201C0054
S113640C80841E0000802500999E360000403800D0
S113641C00093D0000803E0000004B00404B4C0046
S113642C00204E00808D5B0000C05D000080700079
S113643C00127A0000007D0080969800001BB700C3
S113644C0080BB00C0E8CE00647ADA000024F400BB
S113645C0000FA00433A2F576F726B2F736F6674F8
S113646C776172652F4F70656E424C542F54617274
S113647C6765742F44656D6F2F41524D434D335FE7
S113648C4C4D33535F454B5F4C4D33533839363297
S113649C5F43726F7373776F726B732F50726F6786
S11364AC2F6964652F2E2E2F6C69622F64726976A6
S11364BC65726C69622F73797363746C2E6300005C
S11364CC433A2F576F726B2F736F667477617265D3
S11364DC2F4F70656E424C542F5461726765742F44
S11364EC44656D6F2F41524D434D335F4C4D3353C7
S11364FC5F454B5F4C4D3353383936325F43726FC3
S113650C7373776F726B732F50726F672F69646537
S113651C2F2E2E2F6C69622F6472697665726C69EA
S113652C622F7379737469636B2E6300433A2F572C
S113653C6F726B2F736F6674776172652F4F706512
S113654C6E424C542F5461726765742F44656D6FA1
S113655C2F41524D434D335F4C4D33535F454B5F8D
S113656C4C4D3353383936325F43726F7373776FD4
S113657C726B732F50726F672F6964652F2E2E2FD9
S113658C6C69622F6472697665726C69622F7561CD
S113659C72742E6300000000433A2F576F726B2FF6
S11365AC736F6674776172652F4F70656E424C54CD
S11365BC2F5461726765742F44656D6F2F41524D72
S11365CC434D335F4C4D33535F454B5F4C4D33530D
S11365DC383936325F43726F7373776F726B732F04
S11365EC50726F672F6964652F2E2E2F6C69622F82
S11365FC6472697665726C69622F63616E2E6300D6
S903419B20
